:10000000C32800308A000408840A820700340034C0
:10001000763416341E34263425342E3436343D34AA
:100020003E34463445344E3455346A3466340D34E7
:1000300015341D3424342D342C3435343C344334BD
:1000400044344D3454345B345A341C341B3423341C
:100050002B34343433343B3442344B344C34523408
:100060005D341A34223421342A34323431343A346F
:10007000413449344A3451342934EC34F134FA34BB
:10008000FD34E934EB34F534F434F2347734CA34E3
:100090007C347B346C3475347D3479346B34733414
:1000A00074344E34693472347A34DA34703441340E
:1000B000713467347E3400341134673464349134DD
:1000C000AF347834073477345834F0349F340E34F6
:1000D000FF34FE340534063404340C3403340B345A
:1000E00083340A3401340934003400340034593480
:1000F000143400340034003400340034003400344C
:0E010000003400340034003400340034003485
:10017A00D4200F21C9201F22BF2800289F01A001D7
:10018A00A1019E018301BD2883120515CC28822175
:10019A000318D028D128CC288312210808000B3054
:1001AA0083128E001C308D0063308C008C0BDB2890
:1001BA008D0BDB288E0BDB286400080083120615E2
:1001CA0009308C008C0BE728EA28831206141A30AF
:1001DA008C008C0BEE2864008312061006308C000B
:1001EA008C0BF528640008008312061109308C0074
:1001FA008C0BFD280029831206141A308C008C0BF4
:10020A00042964008312061006308C008C0B0B291B
:10021A00640008002521803055210430831294009F
:10022A000930930034309200920B1929930B192943
:10023A00940B19292029FF305521AA30C32108001F
:10024A008B018830831681008312851406100611EB
:10025A0083160514851005110610861406118615D5
:10026A0083129E11FE308C000C08A0000800063094
:10027A0083128C008C0B3F29640083121E12861D88
:10028A0047291E16831206141A308C008C0B4B2930
:10029A006400831206100D308C008C0B5229080062
:1002AA0083128F0009308C000C088E008510A5304F
:1002BA008C005F298C0B5E2983120F186529682927
:1002CA00831285146A29831285100F088C00031083
:1002DA000C0C80388D000D088F00A1308C00752918
:1002EA008C0B74297829013083128E02031D7E2912
:1002FA007F29802981296129080083120518862906
:10030A008729B82985309C009C0B892964008312AF
:10031A00051890299129B82908309C001C089D00CD
:10032A00CF309C0064009C0B972903108312051898
:10033A000314A10CCC309C0064009C0BA12964001E
:10034A00013083129D02031DAB29AC29AD29AE29C8
:10035A009A290518B129B229B5290314C229B8293D
:10036A0005110310C229861CBB29BC29C12986197B
:10037A00BF29C029C1291F2382290800831291009D
:10038A001108FE3A0319CA29CB29CF2911088D0071
:10039A000D08A00006100611861CD429D529D629D5
:1003AA00D729D1298619DA29DB29DC291B2AE32056
:1003BA00831290010314900D08308D000D088F00F0
:1003CA008618E829E929EA291B2A1118ED29EE29B4
:1003DA00F029E320F629F920013083128D000D0857
:1003EA00900711088D0003100D0C8E000E08910065
:1003FA0001308F02031D022A032A042A052AE5294D
:10040A008618082A092A0A2A1B2A10180D2A0E2ACF
:10041A00102AE320112AF920F9208312861C162AB1
:10042A00172A182A192A122A03141E2A0610061134
:10043A00031008008312930013087F39013E8400D9
:10044A0001209200120894008F2A9B2A931B2E2ABD
:10045A002F2A3E2A9E19322A332A372AE030C3210C
:10046A001230C32183129E15E030C3217C30C32190
:10047A004C2A83129E11E030C321F030C3217C3014
:10048A00C321E030C321F030C3211230C3219B2A9B
:10049A008312931B512A522A632AE130C321143052
:1004AA00C3217730C321E130C321F030C321143096
:1004BA00C321F030C3217730C321632A9B2A8312D8
:1004CA00941B682A692A762A931B6C2A6D2A702A39
:1004DA001408C321752AF030C32183121408C321DA
:1004EA008D2A831214087F39920012089400931BF4
:1004FA007F2A802A862AE030C32183121408C32166
:10050A008D2AE030C321F030C32183121408C3219D
:10051A009B2A9B2A83121408003A03192A2AFE3AB4
:10052A0003192B2A013A03194D2A642A08000430B8
:10053A008312920012089300061106109E101E10D4
:10054A001E11A6309200920BA82A64008312861DFF
:10055A00AF2AB02AB22A03101E2B9E148618B62A76
:10056A00B72AB92A03101E2B94010314940D0930DB
:10057A009200120895003C2183121E1EC52AC62A23
:10058A00CA2A013092001208940703101E1A031493
:10059A009F0C8618D12AD22AD42A03101E2B013086
:1005AA009502031DD92ADA2ADB2ADC2AC02A3C2131
:1005BA00013083121405920000301E1A013012060F
:1005CA00031DE82AE92AEA2A9E108619ED2AEE2A4C
:1005DA00022B1E14FF309200120895003C21831250
:1005EA001E1EF82AF92AFA2A022B01309502031D47
:1005FA00FF2A002B012B022BF32AE3208312061178
:10060A009E18082B092B0D2B1E1C0C2B0D2B172BA0
:10061A0001309302031D122B132B142B1D2BFE30BA
:10062A00C321A12A83121E1585309200920B1B2B1F
:10063A00031408009C22031C232B242BFD2B83125A
:10064A001E1D282B292BFD2BDE2BFA30C321031C60
:10065A002F2B302B312B2521FC2BEE30C321FC2BE9
:10066A00FA30C321FC2BFA30C321031C3D2B3E2B4D
:10067A00462BAB30C321031C432B442B462B833020
:10068A00C321FE30831296001608A000FC2B200816
:10069A00C321FC2BFA30C3218312861C552B562BFF
:1006AA006B2B861D592B5A2B6B2BF9309600640045
:1006BA00960B5C2B602B64008312861C652B662BC1
:1006CA006B2B861D692B6A2B6B2B0F21FC2BFA30A7
:1006DA00C3212521FC2BFA30C3219C22031C762B33
:1006EA00772BA62B83121F08F03903197D2B7E2B3B
:1006FA007F2B292B1F08960002300310960CFF3E11
:10070A00031D822B16080139970003300310970D39
:10071A00FF3E031D8B2B1F0898000310180C01398C
:10072A00990002300310990DFF3E031D972B1F08F5
:10073A0001399A001A0719041704FF3A5521FA30A9
:10074A00C321FE30831296001608A000FC2BFA3053
:10075A00C3219C22031CB22BB32BD42B83129F1FC1
:10076A00B72BB82BB92B292B1F08960016089B000C
:10077A001F08960003300310960CFF3E031DC02B82
:10078A0016080C39013E6038552183121B08960061
:10079A000310160C0F3970385521FA30C321FE3078
:1007AA00831296001608A000FC2BFE30C321FC2BF6
:1007BA00FC2B83121F08ED3A0319702B033A031915
:1007CA00322B1C3A0319382B013A0319AC2B073A7E
:1007DA000319352B013A03192A2B033A03196C2BF7
:1007EA00083A03194C2B013A03194F2BDA2BFF2B2A
:0607FA00FE30C3210800DF
:02400E00F23F7F
:00000001FF
